:1000000012C0189572C218951895189518951895DC
:100010001895189518951895189518951895189578
:100020001895189518958FE58DBFC0E4E8E34E2E1E
:1000300084E08EBFD4E0F4E05F2EEEEFF3E0A0E6C4
:10004000B0E088278D933197E9F7E0D2662480EC01
:1000500081BB8FE382BB85B7837F846085BF8FE3DD
:1000600087BBEAE7F0E080E419D358E0C895802D1B
:100070000FD331965A95D1F704C020040C1F0C04FD
:100080002020A7D2EAE3F8E098D2A1D2E4E4F8E095
:1000900094D2E1E0F0E0B1D28BB780688BBF789466
:1000A000D8D10027ADE7B0E08C9181FB0EF401E0E0
:1000B00041E0041709F015C080917D008D7F809389
:1000C0007D0080917D008E7F80937D0080917D00FA
:1000D000806180937D0080917D008F7D80937D0085
:1000E0005FD00027ADE7B0E08C9180FB0EF401E01B
:1000F00041E0041709F015C080917D008D7F809349
:100100007D0080917D008E7F80937D0080917D00B9
:100110008F7E80937D0080917D00806280937D0042
:100120003FD00027A0E3B0E08C9184FB0EF401E007
:1001300040E0041709F030C0ADE7B0E08C9182FBDD
:10014000882780F9809580FBADE7B0E08C9182F93B
:100150008C930027ADE7B0E08C9182FB0EF401E0B8
:1001600040E0041709F00AC08FEB18E041D2EEE43A
:10017000F8E023D28FE718E03BD209C08FE718E000
:1001800037D2EEE4F8E019D28FEB18E031D280E0FC
:100190007FD288EC90E0AED285E090E0ABD281CF08
:1001A0000027ADE7B0E08C9182FB0EF401E040E067
:1001B000041709F048C00027ADE7B0E08C9185FB3B
:1001C0000EF401E041E0041709F005C0A9E7B0E032
:1001D0008C9181508C9300917900013008F003C01C
:1001E00080E1809379000027ADE7B0E08C9184FB3B
:1001F0000EF401E041E0041709F005C0A9E7B0E002
:100200008C918F5F8C9300917900003110F009F090
:1002100001C003C081E08093790040917900009192
:100220007A00041709F405C08091790080937A0060
:1002300076D08FEB18E0DCD1EEE4F8E0BED18FE7AA
:1002400018E0D6D162C00027ADE7B0E08C9185FB05
:100250000EF401E041E0041709F005C0ABE7B0E09F
:100260008C9181508C9300917B00013008F003C089
:1002700080E280937B000027ADE7B0E08C9184FBA7
:100280000EF401E041E0041709F005C0ABE7B0E06F
:100290008C918F5F8C9300917B00003210F009F0FD
:1002A00001C003C081E080937B0040917B000091FE
:1002B0007C00041709F420C080917B0080937C00AF
:1002C00080917B00A9E7B0E0AD90BB24A6E6B0E04A
:1002D000AA0DBB1D8C93A9E7B0E0EC91FF27A9E71D
:1002E000B0E0AD90BB24A6E6B0E0AA0DBB1D91E046
:1002F0007BE78BD253D024D08FE718E079D1EEE49E
:10030000F8E05BD18FEB18E073D1E1E1F0E0A9E711
:10031000B0E091E07BE779D280E0BAD108958FE731
:1003200016E066D1009179000A3008F003C0EEE4CF
:10033000F8E043D1A0E2B4E0E9E7F0E013D235D130
:100340008FEB16E055D1A9E7B0E0AD90BB24A6E64F
:10035000B0E0AA0DBB1D0C910A3008F003C0EEE41A
:10036000F8E02BD1A0E2B4E0E9E7F0E0A190BB24F3
:10037000E6E6F0E0EA0DFB1DF5D117D1A9E7B0E004
:10038000AD90BB24A6E6B0E0AA0DBB1D8C91809376
:100390007B0080917B0080937C000895C198C49A73
:1003A000C29A80E1809362004091620001E00417EC
:1003B00010F009F042C0A2E6B0E0AD90BB24A6E682
:1003C000B0E0AA0DBB1D0C9141E0041BA4E6B0E017
:1003D0000C9391E0A4E6B0E09CD18091640080642D
:1003E0008093640080916400806880936400BD9A6B
:1003F000B89AC09AA4E6B0E0119697E08E91983032
:1004000018F4392F992702C038E09850881FC598F2
:1004100008F4C59A00000000C09800000000C09ACF
:10042000000000003A9591F7992341F7809162000E
:1004300081508093620008F0B7CFC498EF93FF9388
:10044000E0E1F0E04BD1FF91EF91C49AC29AC198DC
:100450000895C198C49AC29A80917D008F7B809341
:100460007D0080917D008F7780937D00C39A81E02D
:100470008093620000916200023110F009F015C013
:10048000A2E6B0E0EC91FF27A2E6B0E0AD90BB247D
:10049000A6E6B0E0AA0DBB1D91E0C8D1A2E6B0E08F
:1004A0008C918F5F8C9308F4E5CF809177008093D7
:1004B0007900A8E7B0E08C9180FBADE7B0E08C91CB
:1004C00082F98C936BDF85D07ED0E0E5F8E075D0C3
:1004D0008FEB11E08DD0E6E5F8E06FD020DF8FE7FD
:1004E00018E086D080E0D4D008950F921F922F920A
:1004F0003F924F925F927F92AF92BF920F931F9362
:100500002F933F934F935F936F937F938F939F931B
:10051000AF93BF93CF93DF93EF93FF938FB78F93F7
:100520000027A0E3B0E08C9183FB0EF401E04427A8
:10053000A0E3B0E08C9182FB0EF44395041709F020
:100540000BC080917D00816080937D0080917D0053
:100550008D7F80937D000AC080917D0082608093B2
:100560007D0080917D008E7F80937D0081E090E012
:10057000C1D08F918FBFFF91EF91DF91CF91BF914C
:10058000AF919F918F917F916F915F914F913F912B
:100590002F911F910F91BF90AF907F905F904F90E0
:1005A0003F902F901F900F901895A0E2B4E08D918E
:1005B000882311F06DD0FBCF0895B3D0802D11F0BA
:1005C00067D0FBCF089582E069D01DD013C080ECC6
:1005D00065C081E063D017D080E860C08FE721302C
:1005E00039F08FEB223021F08FE8233009F08FECC7
:1005F000810F54C080E852D0089588EE93E07AD0FD
:100600003197D9F7089583E0992774C08AEF90E075
:1006100071D0A59AA49AA39AA29AA19AA09AA898EE
:1006200085E090E067D0A998AD98AC98AB9AAA9A6B
:10063000A99AEF93FF93E4ECF0E050D0FF91EF9193
:10064000A99855D0A99AEF93FF93E4ECF0E046D037
:10065000FF91EF91A9984BD0A99AEF93FF93E4EC07
:10066000F0E03CD0FF91EF91A99841D0AA98A99AC7
:10067000EF93FF93E4ECF0E031D0FF91EF91A99874
:1006800036D088E20BD08EE009D086E007D00895FE
:10069000A89A829505D004D02AD00895A898F9CFB9
:1006A000859510F4AA9A01C0AA98859510F4AB9A82
:1006B00001C0AB98859510F4AC9A01C0AC988595B3
:1006C00010F4AD9A01C0AD98A99AEF93FF93E4ECB2
:1006D000F0E004D0FF91EF91A99808953197F1F7D8
:1006E0000895689462F80895E89462F8089581E0A6
:1006F00090E000C0EF93FF93EE27E82BE92B31F059
:10070000E0EDF7E03197F1F70197D1F7FF91EF9125
:100710000895903029F08C91880F9A95E9F78C9381
:100720000895C895319600200895000F111F221FCB
:10073000331F089500951095209530950F5F1F4F3A
:100740002F4F3F4F0895019110810EC001911191DB
:10075000219130810BC00191108117FF05C03FEF3F
:100760002FEF04C0008111272227332737FF03C052
:10077000E1DF8DE28D93CF93DF93CF92DF92EF9203
:10078000AA24BB24CC24DD24EE2440E2CAE0DD27E9
:1007900055E093E38881890F87FD9F7083FD907FEB
:1007A000891B89935A95A9F7C0DFAA1CBB1CCC1CD6
:1007B000DD1CEE1C4A9551F7E894EFE0FF2782918B
:1007C0000ED0EB30E0F71EF068948A2D0CD088270D
:1007D0008D93EF90DF90CF90DF91CF910895982F78
:1007E000829501D0892F8F70805D26F0803309F4C7
:1007F000089568948D930895E199FECFEEBBFFBBF9
:100800003196089591E001C092E07B3751F47FB7B3
:10081000F894F2DF8D918DBBE29AE19A9A95C9F72F
:100820007FBF7727089591E001C092E0E5DFE09A6D
:100830008DB38D939A95D1F708954D415820343357
:1008400035370000314D464B205631630000200003
:0C0850004F55543A2000494E3A20200039
:00000001FF
